:100000000C947B040C9496040C9496040C94960423
:100010000C9496040C9496040C9496040C949604F8
:100020000C9496040C9496040C9496040C949604E8
:100030000C94BA050C9496040C9496040C949604B3
:100040000C9496040C9496040C94D5090C94CD0F42
:100050000C9429070C9496040C9496040C94960422
:100060000C9496040C9496040C9496040C949604A8
:10007000083B3BD74ABC846E023D2FC1FEBD9A317E
:10008000743DDA3D83BE117FC73E4CBBE5BEAAAAD4
:100090006C3F80000000555000000555000A955047
:1000A00000000552000AA5500000054A000AA950A8
:1000B0000000052A000AAA50000004AA000AAA901B
:1000C000000004AA000AAAA0000002AA000AAAA826
:1000D00000000AAA000A6AA800000AAD000A5AA88D
:1000E00000000AB5000A56A800000AD5000A55A863
:1000F00000000B55000A556800000D55000A5550C8
:1001000000000555000AE00000000001000A5A0046
:1001100000000005000A54A000000015000A550A5E
:1001200000000055000A5540A0000155000A555036
:100130000A000555000A555400A01555000A5555EA
:10014000000A5555000A55554001F555000A555508
:1001500050055F55000A5555541555F5000A55557B
:100160005555555F000A40000000000000031000D4
:100170000000000000030400000000000003010074
:100180000000000000030040000000000003001019
:100190000000000000030004000000000003000154
:1001A0000000000000030000400000000003000009
:1001B0001000000000030000040000000003000025
:1001C00001000000000300000040000000030000E8
:1001D0000010000000030000000800000003000001
:1001E0000002000000030000000080000003000087
:1001F00000002000000300000000080000030000D1
:100200000000020000030000000000800003000066
:1002100000000020000300000000000800030000B0
:100220000000000200030000000000008003000046
:100230000000000020030000000000000803000090
:100240000000000004034000000000000003100054
:100250000000000000030400000000000003010093
:100260000000000000030040000000000003001038
:100270000000000000030004000000000003000173
:100280000000000000030000400000000003000028
:100290001000000000030000040000000003000044
:1002A0000100000000030000004000000003000007
:1002B0000010000000030000000800000003000020
:1002C00000020000000300000000800000030000A6
:1002D00000002000000300000000080000030000F0
:1002E0000000020000030000000000800003000086
:1002F00000000020000300000000000800030000D0
:100300000000000200030000000000008003000065
:1003100000000000200300000000000008030000AF
:100320000000000004030000000000000103400082
:1003300000000000000310000000000000030400A3
:100340000000000000030100000000000003004066
:100350000000000000030010000000000003000483
:100360000000000000030001000000000003000086
:100370004000000000030000100000000003000027
:100380000400000000030000010000000003000062
:100390000040000000030000001000000003000007
:1003A000000800000003000000020000000300003D
:1003B0000000800000030000000020000003000097
:1003C000000008000003000000000200000300001D
:1003D0000000008000030000000000200003000077
:1003E00000000008000300000000000200030000FD
:1003F0000000000080030000000000002003000057
:1004000000000000080300000000000004030000DA
:100410000000000001034000000000000003100085
:1004200000000000000304000000000000030100C1
:100430000000000000030040000000000003001066
:1004400000000000000300040000000000030001A1
:100450000000000000030000400000000003000056
:100460001000000000030000040000000003000072
:100470000100000000030000004000000003000035
:10048000001000000003000000080000000300004E
:1004900000020000000300000000800000030000D4
:1004A000000020000003000000000800000300001E
:1004B00000000200000300000000008000030000B4
:1004C00000000020000300000000000800030000FE
:1004D0000000000200030000000000008003000094
:1004E00000000000200300000000000008030000DE
:1004F0000000000004034000000000000003500062
:10050000000000000003540000000000000355003C
:10051000000000000003554000000000000355509B
:100520000000000000035554000000000003555572
:100530000000000000035555400000000003555521
:1005400050000000000355555400000000035555AD
:100550005500000000035555554000000003555557
:1005600055500000000355555554000000035555E3
:10057000555500000003555555554000000355558D
:100580005555500000035555555554000003555519
:1005900055555500000355555555554000035555C3
:1005A000555555500003555555555554000355554F
:1005B00055555555000355555555555540035555F9
:1005C0005555555550035555555555555403555585
:1005D0005555555555035555555555555403555570
:1005E0005555555550035555555555554003555579
:1005F00055555555000355555555555400035555FA
:100600005555555000035555555555400003555502
:100610005555550000035555555554000003555583
:10062000555550000003555555554000000355558C
:10063000555500000003555555540000000355550D
:100640005550000000035555554000000003555516
:100650005500000000035555540000000003555597
:1006600050000000000355554000000000035555A0
:100670000000000000035554000000000003555026
:10068000000000000003554000000000000355007A
:1006900000000000000354000000000000035000B0
:1006A0000000000000034000000000000003000004
:1006B0000000000000038000000000000203A00012
:1006C000000000000A03A800000000002A03AA009E
:1006D00000000000AA03AA8000000002AA03AAA04A
:1006E0000000000AAA03AAA80000002AAA03AAAAD6
:1006F000000000AAAA03AAAA800002AAAA03AAAA22
:10070000A0000AAAAA03AAAAA8002AAAAA03AAAA17
:10071000AA00AAAAAA03AAAAAA82AAAAAA03AAAA59
:10072000AAAAAAAAAA03AAAAAA82AAAAAA03AAAA9F
:10073000AA00AAAAAA03AAAAA8002AAAAA03AAAA3D
:10074000A0000AAAAA03AAAA800002AAAA03AAAA27
:10075000000000AAAA03AAA80000002AAA03AAA0CF
:100760000000000AAA03AA8000000002AA03AA004F
:1007700000000000AA03A800000000002A03A00057
:10078000000000000A0380000000000002030000D7
:1007900000000000000380000000000002032000B1
:1007A0000000000008030800000000002003020011
:1007B0000000000080030080000000020003002011
:1007C00000000008000300080000002000030002F1
:1007D0000000008000030000800002000003000011
:1007E00020000800000300000800200000030000B3
:1007F00002008000000300000082000000030000EF
:100800000028000000030000000000000003540066
:1008100000000000000A015000000000000A00056E
:1008200040000000000A000015000000000A00005F
:1008300000540000000A000000015000000A0000FF
:1008400000000540000A000000000015000A00003A
:100850000000000A000A0000000000A8000A0000D2
:1008600000000A80000A00000002A000000A000048
:1008700000A80000000A00002A000000000A000A88
:1008800080000000000A02A000000000000AA8008A
:1008900000000000000AC00000000003000A3C0045
:1008A00000000000000A03C000000000000A003C35
:1008B00000000000000A0003C0000000000A000061
:1008C0003C000000000A000003C00000000A000015
:1008D000003C0000000A00000003C000000A000005
:1008E00000003C00000A0000000003C0000A0000F5
:1008F0000000003C000A11241FBECFEFD0E1DEBF94
:10090000CDBF11E0A0E0B1E0E8E4F0E302C0059063
:100910000D92AC38B107D9F712E0ACE8B1E001C0F4
:100920001D92A83DB107E1F70C94B2040C940000AD
:10093000CF93DF93CDB7DEB7E4E2F0E086E08083CB
:10094000EAE2F0E01082EBE2F0E080E38083E7E2AD
:10095000F0E08CEF8083E1E2F0E08FEF8083DF91C5
:10096000CF910895CF93DF93CDB7DEB722970FB61F
:10097000F894DEBF0FBECDBF0E9498040E94AB0565
:100980000E9465060E94C00989E29CE09093BD0127
:100990008093BC018CE79CE09093BF018093BE01E3
:1009A00082E29DE09093C1018093C00188EA9DE0BE
:1009B0009093C3018093C2018DE19EE09093C501A5
:1009C0008093C40183E89EE09093C7018093C601A1
:1009D00083E89EE09093C9018093C8011A8219822E
:1009E00011C029813A8189819A81FC01E25FFE4F21
:1009F0008081F901E759FD4F808389819A810196B1
:100A00009A83898389819A818730910554F37894F8
:100A1000A5E2B0E0E5E2F0E0808184608C93809113
:100A200098018823E1F310929801A5E2B0E0E5E295
:100A3000F0E0808182608C93F8941A82198211C050
:100A400029813A8189819A81FC01E050FF4F8081A0
:100A5000F901E759FD4F808389819A8101969A8334
:100A6000898389819A818730910554F378948091A4
:100A700098018823E1F3109298011A82198211C01B
:100A800029813A8189819A81FC01E95FFE4F808149
:100A9000F901E759FD4F808389819A8101969A83F4
:100AA000898389819A818730910554F380919801D7
:100AB0008823E1F310929801A5E2B0E0E5E2F0E0CE
:100AC00080818B7F8C938CE191E00E94D50700C0E0
:100AD00080919C01813011F40E94AF1080919501AA
:100AE000813001F580917A01882369F480919B011E
:100AF0009927880F991FFC01E454FE4F0190F08163
:100B0000E02D09950DC08091930190919401880F7B
:100B1000991FFC01E454FE4F0190F081E02D0995EE
:100B20001092950180919601813031F40E94120F4C
:100B3000109296010E94081080919801813041F630
:100B40000E94A90880919A01813011F40E94030C3F
:100B500010929801BDCFCF93DF93CDB7DEB7E1E818
:100B6000F0E082E48083EFE6F0E080E28083DF91D2
:100B7000CF9108951F920F920FB60F9211242F93C9
:100B80003F934F935F936F937F938F939F93AF9315
:100B9000BF93EF93FF93CF93DF93CDB7DEB78091F1
:100BA0009E0190919F010097B1F4E6E8F0E080810A
:100BB00091819093A5018093A401A1E8B0E0E1E8C0
:100BC000F0E080818F7B8C9381E090E090939F0197
:100BD00080939E0167C0E6E8F0E080819181909368
:100BE000A3018093A201A1E8B0E0E1E8F0E08081F8
:100BF00080648C932091A2013091A3018091A40183
:100C00009091A501A901481B590BCA019093A1011C
:100C10008093A00110929F0110929E018091A001EB
:100C20009091A101845C99409093A1018093A001CF
:100C30008091A0019091A10120E931E0B9010E94C9
:100C40008F16CB019093A1018093A0018091A00108
:100C50009091A101992324F41092A1011092A00176
:100C60008091A0019091A1018730910534F086E038
:100C700090E09093A1018093A0012091A001309178
:100C8000A10180919301909194012817390751F0A7
:100C90001092AF018091A0019091A10190939401D5
:100CA00080939301DF91CF91FF91EF91BF91AF912D
:100CB0009F918F917F916F915F914F913F912F9174
:100CC0000F900FBE0F901F901895CF93DF93CDB765
:100CD000DEB7E0ECF0E01082E1ECF0E088E9808340
:100CE000E2ECF0E086E08083E4ECF0E085E18083F4
:100CF000E5ECF0E01082DF91CF910895CF93DF9380
:100D0000CDB7DEB764970FB6F894DEBF0FBECDBF88
:100D100083E28F83188683E689871A861B8685E09F
:100D200090E09E838D831C821B821A82198215C0DB
:100D300029813A81CE010796FC01E20FF31F8081E1
:100D4000282F33278B819C81820F931F9C838B8359
:100D500089819A8101969A83898329813A818D813B
:100D60009E812817390724F38B819C8120E030E194
:100D7000B9010E94A3169C838B838D819E819A8BDF
:100D8000898B8B819C819C8B8B8B8B899C899923F4
:100D90002CF48B899C89CF969C8B8B8B8B899C891F
:100DA000082E892F000C881F990B000C881F991F93
:100DB000282F235CCE010796E989FA89E80FF91FED
:100DC00020838D819E8101969E838D83ED81FE819E
:100DD0008B819C8120E430E0B9010E94A316282F6A
:100DE000235CCE010796E80FF91F20838D819E8139
:100DF00001969E838D832D813E81CE010796FC0155
:100E0000E20FF31F8DE080838D819E8101969E838A
:100E10008D831A8219820FC029813A81CE010796EB
:100E2000FC01E20FF31F80810E94B50789819A813E
:100E300001969A83898389819A818830910564F328
:100E400064960FB6F894DEBF0FBECDBFDF91CF9191
:100E500008951F920F920FB60F9211242F933F9374
:100E60008F939F93AF93BF93EF93FF93CF93DF93B2
:100E7000CDB7DEB72397DEBFCDBFE6ECF0E08081D3
:100E8000898389818D30C9F48091A6018130A9F4CC
:100E9000A5E2B0E0E5E2F0E080818B7F8C931092D8
:100EA000A60181E080939C01809166029927FC0154
:100EB000E253FE4F8981808345C08091A601282F8F
:100EC00033273B832A838A819B81009731F02A81D3
:100ED0003B812130310511F135C08981833271F4B4
:100EE00080919C01882351F481E08093A601A5E2C2
:100EF000B0E0E5E2F0E0808184608C9310926602BD
:100F000020916602822F9927FC01E253FE4F8981CE
:100F10008083822F8F5F8093660214C08091660267
:100F20009927FC01E253FE4F8981808380916602FC
:100F3000863930F4809166028F5F8093660202C02A
:100F40001092A6012396F894DEBFCDBFDF91CF911A
:100F5000FF91EF91BF91AF919F918F913F912F9111
:100F60000F900FBE0F901F901895CF93DF93CDB7C2
:100F7000DEB721970FB6F894DEBF0FBECDBF8983D1
:100F8000E0ECF0E080819927807290700097C1F3C7
:100F9000E6ECF0E08981808321960FB6F894DEBFFD
:100FA0000FBECDBFDF91CF910895CF93DF93CDB723
:100FB000DEB726970FB6F894DEBF0FBECDBF9E8377
:100FC0008D838D819E81DC01FD0101900020E9F778
:100FD0003197CF018A1B9B0B9C838B831A821982CA
:100FE0000FC029813A818D819E81F901E80FF91F97
:100FF00080810E94B50789819A8101969A838983AD
:1010000029813A818B819C818217930750F78091C7
:1010100037010E94B507809138010E94B5072696D6
:101020000FB6F894DEBF0FBECDBFDF91CF9108950C
:10103000CF93DF93CDB7DEB766970FB6F894DEBFD8
:101040000FBECDBF9E8B8D8B8D899E894AE050E06F
:101050009E012F5F3F4FB9010E945E16CE0101969F
:101060000E94D50766960FB6F894DEBF0FBECDBFBF
:10107000DF91CF910895CF93DF93CDB7DEB76E9711
:101080000FB6F894DEBF0FBECDBF80E489838DE636
:101090008A831B8280917A01813079F482E78B8385
:1010A0002091930130919401CE010B964AE050E0DB
:1010B000BC01C9010E945E160EC088E68B83809138
:1010C0009B01282F3327CE010B964AE050E0BC014C
:1010D000C9010E945E161C82CE010B96DC01FD0147
:1010E00001900020E9F73197CF018A1B9B0B9E01ED
:1010F000255F3F4FAC01B901CE0101960E944E160B
:10110000CE010196DC01FD0101900020E9F7319745
:101110009F012A1B3B0BCE010196820F931FFC01FE
:1011200083E290E091838083CE0101960E94D507EF
:10113000809137010E94B507809138010E94B50760
:101140006E960FB6F894DEBF0FBECDBFDF91CF9184
:101150000895CF93DF93CDB7DEB76E970FB6F894AF
:10116000DEBF0FBECDBF2091980230919902CE0113
:101170000B964AE050E0BC01C9010E945E1680E473
:1011800089838EE48A8380E38B831C82CE010B9655
:10119000DC01FD0101900020E9F73197CF018A1BA6
:1011A0009B0B9E01255F3F4FAC01B901CE0101961B
:1011B0000E944E16CE010196DC01FD010190002037
:1011C000E9F731979F012A1B3B0BCE010196820F55
:1011D000931FFC0183E290E091838083CE0101960E
:1011E0000E94D50720919A0230919B02CE010B9666
:1011F0004AE050E0BC01C9010E945E1680E4898388
:1012000082E58A8381E38B831C82CE010B96DC010D
:10121000FD0101900020E9F73197CF018A1B9B0B5C
:101220009E01255F3F4FAC01B901CE0101960E949E
:101230004E16CE010196DC01FD0101900020E9F778
:1012400031979F012A1B3B0BCE010196820F931F02
:10125000FC0183E290E091838083CE0101960E949D
:10126000D5072091870230918802CE010B964AE083
:1012700050E0BC01C9010E945E1680E4898386E4C7
:101280008A8382E38B831C82CE010B96DC01FD01F5
:1012900001900020E9F73197CF018A1B9B0B9E013B
:1012A000255F3F4FAC01B901CE0101960E944E1659
:1012B000CE010196DC01FD0101900020E9F7319794
:1012C0009F012A1B3B0BCE010196820F931FFC014D
:1012D00083E290E091838083CE0101960E94D5073E
:1012E00020918C0230918D02CE010B964AE050E0A5
:1012F000BC01C9010E945E1680E4898387E78A8366
:1013000081E38B831C82CE010B96DC01FD010190F1
:101310000020E9F73197CF018A1B9B0B9E01255FC7
:101320003F4FAC01B901CE0101960E944E16CE018D
:101330000196DC01FD0101900020E9F731979F0142
:101340002A1B3B0BCE010196820F931FFC0183E207
:1013500090E091838083CE0101960E94D507809111
:1013600037010E94B507809138010E94B5076E963B
:101370000FB6F894DEBF0FBECDBFDF91CF910895B9
:10138000CF93DF93CDB7DEB7A5E4B0E0E5E4F0E0BE
:10139000808182608C93AEE6B0E0EEE6F0E0808182
:1013A00081608C93DF91CF9108951F920F920FB6B9
:1013B0000F9211242F933F938F939F93AF93BF93DB
:1013C000EF93FF93CF93DF93CDB7DEB72297DEBFC6
:1013D000CDBF8091A9019091AA0101969093AA0195
:1013E0008093A9018091A9019091AA018436910569
:1013F00019F581E0809395011092AA011092A9013C
:10140000809170028F5F80937002809170028436A9
:1014100029F41092700281E0809398018091680213
:101420008F5F80936802809168028A3029F410925D
:10143000680281E080939601E3E2F0E080819927E1
:1014400080719070009711F01092B7018091A70100
:10145000282F33273A83298389819A818630910501
:1014600009F4EEC029813A812730310524F58981BC
:101470009A818230910509F47DC029813A81233017
:10148000310564F489819A81009709F43FC029816C
:101490003A812130310509F451C099C189819A817D
:1014A0008430910509F499C029813A8125303105AC
:1014B0000CF0AAC076C089819A818A30910509F41E
:1014C00025C129813A812B3031056CF489819A81BB
:1014D0008830910509F4E7C029813A812930310526
:1014E0000CF0F8C0C4C089819A818C30910509F450
:1014F00040C129813A812C3031050CF41EC189810B
:101500009A818D30910509F44BC161C18091A80188
:101510008F5F8093A8018091A801883008F457C19B
:101520001092A801ABE2B0E0EBE2F0E090818FE72F
:1015300089238C9381E08093A70149C18091A80100
:101540008F5F8093A8018091A801883008F43FC183
:101550001092A801E2E2F0E0809169028083A8E2A3
:10156000B0E0E8E2F0E0808184608C9382E08093D8
:10157000A7012DC18091A8018F5F8093A801809160
:10158000A801883008F423C11092A801A8E2B0E0B5
:10159000E8E2F0E080818B7F8C9383E08093A70169
:1015A00016C18091A8018F5F8093A8018091A80146
:1015B000883008F40CC11092A801E2E2F0E08091BA
:1015C0006A028083A8E2B0E0E8E2F0E0808188600F
:1015D0008C9384E08093A701FAC08091A8018F5F6B
:1015E0008093A8018091A801883008F4F0C010927F
:1015F000A801A8E2B0E0E8E2F0E08081877F8C9368
:1016000085E08093A701E3C08091A8018F5F80935C
:10161000A8018091A801883008F4D9C01092A801CF
:10162000E2E2F0E080916B028083A8E2B0E0E8E2C1
:10163000F0E0808180618C9386E08093A701C7C031
:101640008091A8018F5F8093A8018091A8018830C4
:1016500008F4BDC01092A801A8E2B0E0E8E2F0E012
:1016600080818F7E8C9387E08093A701B0C08091AA
:10167000A8018F5F8093A8018091A801883008F4A9
:10168000A6C01092A801E2E2F0E080916C02808393
:10169000A8E2B0E0E8E2F0E0808180628C9388E02C
:1016A0008093A70194C08091A8018F5F8093A801C7
:1016B0008091A801883008F48AC01092A801A8E29D
:1016C000B0E0E8E2F0E080818F7D8C9389E0809348
:1016D000A7017DC08091A8018F5F8093A8018091B0
:1016E000A801883008F473C01092A801E2E2F0E08B
:1016F00080916D028083A8E2B0E0E8E2F0E08081B2
:1017000080648C938AE08093A70161C08091A801D6
:101710008F5F8093A8018091A801883008F457C09A
:101720001092A801A8E2B0E0E8E2F0E080818F7BAF
:101730008C938BE08093A7014AC08091A8018F5FB2
:101740008093A8018091A801883008F440C01092CD
:10175000A801E2E2F0E080916E028083A8E2B0E0AE
:10176000E8E2F0E0808180688C938CE08093A701B0
:101770002EC08091A8018F5F8093A8018091A8015D
:10178000883028F11092A801A8E2B0E0E8E2F0E089
:1017900090818FE789238C938DE08093A70117C0F8
:1017A0008091A8018F5F8093A8018091A801883063
:1017B00070F01092A801E2E2F0E01082ABE2B0E03B
:1017C000EBE2F0E0808180688C931092A701229672
:1017D000F894DEBFCDBFDF91CF91FF91EF91BF9124
:1017E000AF919F918F913F912F910F900FBE0F90CE
:1017F0001F901895CF93DF93CDB7DEB780919901F5
:10180000DF91CF910895CF93DF93CDB7DEB780916D
:10181000AE01813051F4A5E2B0E0E5E2F0E0808174
:101820008D7F8C931092AE010AC0A5E2B0E0E5E294
:10183000F0E0808182608C9381E08093AE01DF9143
:10184000CF910895CF93DF93CDB7DEB7DF91CF91DE
:101850000895CF93DF93CDB7DEB722970FB6F894F4
:10186000DEBF0FBECDBF8091B2018823F9F4F8949A
:101870001A82198211C029813A8189819A81FC01D9
:10188000E050FF4F8081F901E759FD4F8083898146
:101890009A8101969A83898389819A8187309105FB
:1018A00054F3789481E08093B2011DC0F8941A82B9
:1018B000198211C029813A8189819A81FC01E95FED
:1018C000FE4F8081F901E759FD4F808389819A811C
:1018D00001969A83898389819A818730910554F38F
:1018E00078941092B20122960FB6F894DEBF0FBE24
:1018F000CDBFDF91CF910895CF93DF93CDB7DEB702
:1019000025970FB6F894DEBF0FBECDBFF8941D82A9
:101910001C8225C04C815D8180918E0290918F0246
:10192000880F991F880F991F880F991F9C018C8120
:101930009D81280F391F86E998E0820F931F9B83B2
:101940008A83EA81FB81849189838981FA01E7593D
:10195000FD4F80838C819D8101969D838C838C813A
:101960009D8187309105B4F2789425960FB6F8944E
:10197000DEBF0FBECDBFDF91CF910895CF93DF9330
:10198000CDB7DEB725970FB6F894DEBF0FBECDBF3B
:1019900080917A01813029F48091AF018093B10167
:1019A00004C08091B0018093B1011D821C8224C0CB
:1019B0004C815D818091B1019927880F991F880F13
:1019C000991F880F991F9C018C819D81280F391FB9
:1019D00086E990E0820F931F9B838A83EA81FB81D3
:1019E000849189838981FA01E759FD4F80838C8135
:1019F0009D8101969D838C838C819D81873091058B
:101A0000BCF28091B1018F5F8093B1018091B101EF
:101A10008E3010F01092B10180917A01813029F45A
:101A20008091B1018093AF0104C08091B101809396
:101A3000B00125960FB6F894DEBF0FBECDBFDF9183
:101A4000CF910895CF93DF93CDB7DEB728970FB628
:101A5000F894DEBF0FBECDBF8091390181508093D5
:101A6000390180913901882309F069C080917A0198
:101A7000813029F48091AF018093B10104C080913D
:101A8000B0018093B1018091B1019927880F991F0E
:101A9000880F991F880F991F9C0186E091E0079697
:101AA000820F931F9E838D83ED81FE8184918C83B1
:101AB0008C818093390118861F8224C04F815885FC
:101AC0008091B1019927880F991F880F991F880F5E
:101AD000991F9C018F819885280F391F86E091E01E
:101AE000820F931F9B838A83EA81FB818491898380
:101AF0008981FA01E759FD4F80838F81988501968E
:101B000098878F838F81988587309105BCF280916B
:101B1000B1018F5F8093B1018091B1018C3010F0E1
:101B20001092B10180917A01813029F48091B10144
:101B30008093AF0104C08091B1018093B0012896D9
:101B40000FB6F894DEBF0FBECDBFDF91CF910895E1
:101B5000CF93DF93CDB7DEB722970FB6F894DEBFF1
:101B60000FBECDBF809139018150809339018091A2
:101B70003901882309F058C080917A01813029F415
:101B80008091AF018093B10104C08091B001809336
:101B9000B1018091B1019927880F991F880F991F72
:101BA000880F991FFC01EF5BFE4F80818093390104
:101BB0001A8219821CC049815A818091B1019927EA
:101BC00029813A81880F991F880F991F880F991FC3
:101BD000820F931FFC01E65CFE4F8081FA01E759FA
:101BE000FD4F808389819A8101969A8389838981B7
:101BF0009A8187309105FCF28091B1018F5F8093CB
:101C0000B1018091B101883011F41092B10180913D
:101C10007A01813029F48091B1018093AF0104C031
:101C20008091B1018093B00122960FB6F894DEBF87
:101C30000FBECDBFDF91CF910895CF93DF93CDB786
:101C4000DEB725970FB6F894DEBF0FBECDBF8091EB
:101C50007A01813029F48091AF018093B10104C0F1
:101C60008091B0018093B101F8941D821C8224C040
:101C70004C815D818091AF019927880F991F880F52
:101C8000991F880F991F9C018C819D81280F391FF6
:101C90008EE098E0820F931F9B838A83EA81FB8109
:101CA000849189838981FA01E759FD4F80838C8172
:101CB0009D8101969D838C838C819D8187309105C8
:101CC000BCF278948091AF018F5F8093AF018091D7
:101CD000AF01813110F01092AF0180917A01813013
:101CE00029F48091B1018093AF0104C08091B101CA
:101CF0008093B00125960FB6F894DEBF0FBECDBF1E
:101D0000DF91CF910895CF93DF93CDB7DEB72897BA
:101D10000FB6F894DEBF0FBECDBF80913901815060
:101D20008093390180913901882309F069C080913D
:101D30007A01813029F48091AF018093B10104C010
:101D40008091B0018093B1018091AF019927880FF4
:101D5000991F880F991F880F991F9C0186E691E0B3
:101D60000796820F931F9E838D83ED81FE81849160
:101D70008C838C818093390118861F8224C04F8107
:101D800058858091AF019927880F991F880F991F57
:101D9000880F991F9C018F819885280F391F86E62F
:101DA00091E0820F931F9B838A83EA81FB81849158
:101DB00089838981FA01E759FD4F80838F81988556
:101DC000019698878F838F81988586309105BCF224
:101DD0008091AF018F5F8093AF018091AF01873D0C
:101DE00010F01092AF0180917A01813029F4809136
:101DF000B1018093AF0104C08091B1018093B00123
:101E000028960FB6F894DEBF0FBECDBFDF91CF91FD
:101E10000895CF93DF93CDB7DEB70E94AA11DF916B
:101E2000CF910895CF93DF93CDB7DEB722970FB64A
:101E3000F894DEBF0FBECDBFE9E2F0E080819927C4
:101E4000807290700097B9F58091B3018F5F809395
:101E5000B301A5E2B0E0E5E2F0E0808184608C931C
:101E600081E08093B5018091B301853079F5A5E2D9
:101E7000B0E0E5E2F0E080818B7F8C931092B501B9
:101E800080917A01813041F41092B00110927A0170
:101E900081E080939A011AC081E080937A011092C8
:101EA000AF0110929A01A5E2B0E0E5E2F0E0808196
:101EB00082608C930BC01092B301A5E2B0E0E5E222
:101EC000F0E080818B7F8C931092B501E9E2F0E025
:101ED0008081992780719070009779F580917A01BF
:101EE000882309F046C0A5E2B0E0E5E2F0E0808199
:101EF00084608C9381E08093B6018091B4018F5F00
:101F00008093B4018091B401853099F5A5E2B0E0E9
:101F1000E5E2F0E080818B7F8C931092B601809196
:101F20009B018F5F80939B0180919B01873011F40F
:101F300010929B011092B0011CC01092B4018091CC
:101F4000B5011A82882311F481E08A838091B60159
:101F50001982882311F491E099838A8199818923D8
:101F6000882339F0A5E2B0E0E5E2F0E080818B7FE4
:101F70008C9322960FB6F894DEBF0FBECDBFDF91D3
:101F8000CF910895CF93DF93CDB7DEB7ECE4F0E0C7
:101F900082EC8083DF91CF9108951F920F920FB64C
:101FA0000F9211242F933F938F939F93AF93BF93DF
:101FB000EF93FF93CF93DF93CDB7DEB78091B70157
:101FC00099279C0180917B0190917C01D901A80FF8
:101FD000B91FEEE4F0E080818C938091B7018F5FB0
:101FE0008093B7018091B701883019F487E080931E
:101FF000B701DF91CF91FF91EF91BF91AF919F9189
:102000008F913F912F910F900FBE0F901F901895B9
:10201000EF92FF920F931F93CF93DF93CDB7DEB76D
:1020200080919A0290919B02909581959F4F9093F9
:102030009502809394028091980290919902AA2728
:1020400097FDA095BA2FBC01CD010E94D4137B014E
:102050008C018091940290919502AA2797FDA095FA
:10206000BA2FBC01CD010E94D413DC01CB01A80121
:102070009701BC01CD010E94ED16DC01CB018093DC
:10208000900290939102A0939202B0939302809158
:10209000900290919102A0919202B091930220E05F
:1020A00030E044E353E4BC01CD010E94FC11DC01AB
:1020B000CB017C018D0180917D0190917E01A091E9
:1020C0007F01B09180019C01AD01C801B7010E9460
:1020D0001A13DC01CB01BC01CD010E943D14DC01CF
:1020E000CB0190938D0280938C0280918C02909111
:1020F0008D02992354F480918C0290918D0288591D
:102100009E4F90938D0280938C0280918C029091CF
:102110008D022EE130E0B9010E94A316CB0190930D
:102120008F0280938E0280918E0290918F0299236C
:1021300024F410928F0210928E0280918E02909160
:102140008F028C30910524F010928F0210928E0233
:10215000DF91CF911F910F91FF90EF900895CF9352
:10216000DF93CDB7DEB764970FB6F894DEBF0FBE2E
:10217000CDBF83E090E09C8B8B8B1A82198283E920
:1021800090E09C838B8310929C018091D0018434D9
:1021900009F0D7C0CFC08B899C89FC01E253FE4F68
:1021A00080819927CD979A8B898B8B899C89019601
:1021B0009C8B8B8B8B899C89FC01E253FE4F808129
:1021C0009927CD97988B8F878B899C8901969C8BBB
:1021D0008B8B8B899C89FC01E253FE4F8081992770
:1021E000CD979E878D878B899C8901969C8B8B8B45
:1021F0008B899C89FC01E253FE4F80819927CD9702
:102200009C878B878B899C8901969C8B8B8B89897A
:102210009A899C01220F331F220F331F8F859889C3
:102220009595879595958795959587959595879596
:10223000822B932B9A8789878F8598898F709070CE
:102240009C0122953295307F3227207F32278D8561
:102250009E859595879595958795822B932B988745
:102260008F838D859E85837090709C0100243695A8
:1022700027950794369527950794322F202D8B8527
:102280009C85822B932B9E838D838B819C810197D0
:102290009C838B838B819C812FEF8F3F920709F466
:1022A0004EC089819A819C01809181019091820127
:1022B000F901E80FF91F8985808389819A81019648
:1022C0009A8389838B819C8101979C838B838B81EB
:1022D0009C812FEF8F3F920791F189819A819C0118
:1022E0008091810190918201F901E80FF91F8F819E
:1022F000808389819A8101969A8389838B819C81CD
:1023000001979C838B838B819C812FEF8F3F92075A
:10231000B1F089819A819C01809181019091820123
:10232000F901E80FF91F8D81808389819A810196D7
:102330009A8389838B819C81009709F02CCF0E941E
:10234000AA1164960FB6F894DEBF0FBECDBFDF9121
:10235000CF910895CF93DF93CDB7DEB78091A202DE
:102360009091A3029093650280936402209164028D
:10237000309165028091CA019091CB01A901481B5F
:10238000590BCA019093BB018093BA0180916402FA
:10239000909165029093CB018093CA012091B8017E
:1023A0003091B9018091BA019091BB01820F931FC6
:1023B0009093B9018093B80180919D018F5F8093C4
:1023C0009D0180919D018630A1F410929D01809124
:1023D000B8019091B90125E030E0B9010E94A3163F
:1023E000CB019093CD018093CC011092B901109252
:1023F000B801DF91CF910895A0E2B0E0E2E0F2E110
:102400000C94B61669837A838B839C832D833E83D9
:102410004F8358878E01075E1F4FB801CE0101968A
:102420000E94AF15F1E1EF2EF12CEC0EFD1EB7016D
:10243000CE0105960E94AF15898D823078F099897A
:10244000923040F420E09A8D8A89981321E02A8BFB
:10245000B701E9C0843051F4923061F020E09A8DE8
:102460008A89981321E02A8FB801DDC0943029F4BD
:10247000823041F763E871E0D6C0823079F3923060
:1024800009F32D8D3E8D4F8D58A18D899E89AF8981
:10249000B88D222433242101AA24BB246501EE2413
:1024A000FF24870160E070E00DC06F5F7F4F6032F6
:1024B000710599F1880F991FAA1FBB1F5695479563
:1024C0003795279520FF19C0280E391E4A1E5B1E1E
:1024D000662477244301281639064A065B0628F449
:1024E000E1E06E2E712C812C912CAE0CBF1CC01E15
:1024F000D11EA60CB71CC81CD91CEE0CFF1C001F5B
:10250000111FB7FFD2CFE1E06E2E712C812C912CE0
:10251000E628F72808291929C8CF8B8D9C8D2B898F
:102520003C89820F931F02969C878B871A869A8D0F
:102530008A89981711F081E08A87D7FE17C08B85AA
:102540009C85A0FE0CC0569447943794279420E0B5
:1025500030E040E050E8222A332A442A552AD69413
:10256000C794B794A79401969C878B8730E0A316F5
:1025700030E0B30630E0C30630E4D30618F58B85AF
:102580009C850EC0220C331C441C551C019720E076
:10259000A21620E0B20620E0C20620E4D20680F4B3
:1025A000AA0CBB1CCC1CDD1C57FEECCF31E0632E0B
:1025B000712C812C912CA628B728C828D928E2CFC5
:1025C0009C878B87D601C5018F779070A070B07003
:1025D00080349105A105B10551F0AD86BE86CF8648
:1025E000D88A83E08987BE01675F7F4F1CC0A7FC44
:1025F000F4CF211431044104510479F380E490E0D4
:10260000A0E0B0E0A80EB91ECA1EDB1E80E8682E4E
:102610008FEF782E8FEF882E8FEF982EA620B72081
:10262000C820D920DACFCB010E948D14E2E1A09618
:102630000C94D216A8E1B0E0E0E2F3E10C94BC16F1
:1026400069837A838B839C832D833E834F83588752
:10265000B1E18B2E912C8C0E9D1EB401CE01019602
:102660000E94AF158E01075F1F4FB801CE0105967E
:102670000E94AF152989223008F46AC039853230AA
:1026800008F468C08A899A8589278A8B243009F4DE
:1026900063C0223009F460C0343041F41D8A1E8AC0
:1026A0001F8A188E1C8A1B8AB40177C0323009F445
:1026B00058C06B897C898B859C85681B790B7C8BCA
:1026C0006B8B2D893E894F89588DED84FE840F8553
:1026D00018892E153F054007510740F4220F331F7C
:1026E000441F551F615070407C8B6B8B80E090E0E5
:1026F000A0E0B0E4AA24BB24650160E070E02E15E0
:102700003F054007510740F0A82AB92ACA2ADB2A08
:102710002E193F09400B510BB695A79597958795B4
:10272000220F331F441F551F6F5F7F4F6F3171059D
:1027300031F7D601C5018F779070A070B0708034EA
:102740009105A105B10589F0AD8ABE8ACF8AD88EE0
:10275000B40123C0B80121C03217D1F763E871E09A
:102760001CC084E0898BB40118C0A7FCEDCF2115F3
:1027700031054105510541F380E490E0A0E0B0E06F
:10278000A80EB91ECA1EDB1E80E89FEFAFEFBFEF99
:10279000A822B922CA22DB22D7CFCB010E948D14F6
:1027A000ECE068960C94D816A8E0B0E0EAEDF3E10E
:1027B0000C94C5169B01AC0183E089831A8257FDF6
:1027C00051C0211531054105510539F482E0898355
:1027D000CE0101960E948D144CC0EEE1F0E0FC8326
:1027E000EB838A818823C9F1203010E0310710E0A3
:1027F000410710E85107C9F188279927DC01821B9E
:10280000930BA40BB50B8D839E83AF83B8872D816B
:102810003E814F815885203080E0380780E04807AE
:1028200080E45807A8F6EB81FC81DA01C901880F22
:10283000991FAA1FBB1F31979C01AD01803010E08A
:10284000910710E0A10710E4B10778F3FC83EB8354
:102850008D839E83AF83B887BBCF2D833E834F8309
:102860005887D5CF81E08A83ACCF60E070E080E00C
:102870009FECE3E028960C94E116ACE0B0E0E3E4D2
:10288000F4E10C94C61669837A838B839C83BE0122
:102890006B5F7F4FCE0101960E94AF158D81823014
:1028A00061F0823050F0843069F48E81882359F5CC
:1028B0002FEF3FEF4FEF5FE72AC020E030E040E02E
:1028C00050E025C02F81388537FDF7CF2F313105F6
:1028D00064F78EE190E0821B930B29853A854B8546
:1028E0005C8504C056954795379527958A95D2F70C
:1028F0008E81882361F050954095309521953F4F0A
:102900004F4F5F4F04C020E030E040E050E8CA0184
:10291000B901E2E02C960C94E2164F925F926F920E
:102920007F928F929F92AF92BF92DF92EF92FF922F
:102930000F931F9320E030E040E050E0FC01E48082
:10294000F58006811781D1808081823038F4D801EA
:10295000C701A061AF77B0706FEFD9C0843009F4C0
:102960006EC0823009F471C0E114F1040105110553
:1029700009F46BC0828193816FEF823896070CF067
:102980006AC062E87FEF681B790B6A3171050CF051
:1029900080C047015801062E04C0B694A7949794AE
:1029A00087940A94D2F744245524320181E090E0C0
:1029B000A0E0B0E004C0880F991FAA1FBB1F6A9552
:1029C000D2F70197A109B109E822F9220A231B23B2
:1029D000E114F1040105110529F061E0462E512CA6
:1029E000612C712C85017401E428F528062917292A
:1029F000D801C7018F779070A070B07080349105B6
:102A0000A105B10509F457C0D801C701CF96A11D92
:102A1000B11D60E070E08030E0E09E07E0E0AE07CE
:102A2000E0E4BE0710F061E070E027E0B695A795FE
:102A3000979587952A95D1F7AF77B07068C080E0F9
:102A400090E0A0E0B0E06FEF62C080E090E0A0E036
:102A5000B0E060E05CC0803891058CF7BC01615843
:102A60007F4FD801C7018F779070A070B07080340D
:102A70009105A105B105A1F08FE390E0A0E0B0E0E1
:102A8000E80EF91E0A1F1B1F17FD28C0D801C70139
:102A9000CCCF60E070E080E090E0A0E0B0E0CCCF90
:102AA000E7FEF2CF80E490E0A0E0B0E0E80EF91E8F
:102AB0000A1F1B1FE9CFE7FC18C080E090E060E030
:102AC000E61660E0F60660E0060760E4160710F020
:102AD00081E090E0BC01D801C701A7CF169507950A
:102AE000F794E7946F5F7F4FD1CFD801C701805C27
:102AF0009F4FAF4FBF4F60E070E08030E0E09E0737
:102B0000E0E0AE07E0E4BE0708F48FCF8CCF282FBB
:102B1000392F9A2F9F77842F8078892B962F97951E
:102B2000992797958F77482F492B6695852F807821
:102B3000862BD794DD24D7948F77582F5D29CA012F
:102B4000B9011F910F91FF90EF90DF90BF90AF9070
:102B50009F908F907F906F905F904F900895FC01B1
:102B6000DB01208131819281492F4F7750E0991FFD
:102B70009927991F8381682F660F692B881F8827E3
:102B8000881FFD018183662309F049C021153105A5
:102B90004105510509F470C082E89FEFFD01938360
:102BA0008283220F331F441F551F220F331F441FE0
:102BB000551F220F331F441F551F220F331F441F61
:102BC000551F220F331F441F551F220F331F441F51
:102BD000551F220F331F441F551F83E08C93203055
:102BE000F0E03F07F0E04F07F0E45F0790F482E881
:102BF0009FEF220F331F441F551F0197203060E0C5
:102C0000360760E0460760E4560798F3FD019383BA
:102C10008283FD01248335834683578308956F3F64
:102C200071F1862F99278F579040FD0193838283FE
:102C300083E08C93220F331F441F551F220F331F35
:102C4000441F551F220F331F441F551F220F331FD0
:102C5000441F551F220F331F441F551F220F331FC0
:102C6000441F551F220F331F441F551F50642483D8
:102C7000358346835783089582E08C930895211508
:102C800031054105510519F484E08C93089544FD04
:102C900002C01C92BECF81E08C93BBCFFB01DC0154
:102CA0000D900020E9F711974150504028F0019015
:102CB00000200D92C9F708951C920895FB019F0111
:102CC000E8944230C4F04532B4F44A3029F497FB1A
:102CD0001EF4909581959F4F642F77270E948F1641
:102CE000805D8A330CF0895D8193CB010097A1F759
:102CF00016F45DE251931082C9010C947F16DC0139
:102D0000FC0101900020E9F73297AE17BF0730F4BD
:102D10007C916081708331976D93F7CF0895AA1BE2
:102D2000BB1B51E107C0AA1FBB1FA617B70710F0B6
:102D3000A61BB70B881F991F5A95A9F780959095E8
:102D4000BC01CD01089597FB092E07260AD077FD17
:102D500004D0E5DF06D000201AF4709561957F4F0E
:102D60000895F6F7909581959F4F08952F923F9281
:102D70004F925F926F927F928F929F92AF92BF928B
:102D8000CF92DF92EF92FF920F931F93CF93DF9337
:102D9000CDB7DEB7CA1BDB0B0FB6F894DEBF0FBE94
:102DA000CDBF09942A88398848885F846E847D84E1
:102DB0008C849B84AA84B984C884DF80EE80FD80E3
:102DC0000C811B81AA81B981CE0FD11D0FB6F89459
:102DD000DEBF0FBECDBFED010895552319F0992335
:102DE00051F018C09923A1F097FB6BED7FE089ECBF
:102DF0009FE397F90895552359F02AF46BED7FE08E
:102E000089E490E40895662777278827992708950D
:102E10000C9420171F93112797FD116057FD126026
:102E20000E941A130E94661711FF08C02BED3FE0A5
:102E300049E450E410FD50680E9424171F91089542
:102E40009FEF80EC08955058192EC7D001D07AC05A
:102E5000BA176207730784079507B1F188F40EF477
:102E600010940B2EBA2FA02D062E622F202D072E88
:102E7000732F302D082E842F402D092E952F502D85
:102E8000FF275523B9F0591B49F0573E98F0469556
:102E900037952795A795F0405395C9F776F0BA0F67
:102EA000621F731F841F30F4879577956795B795D8
:102EB000F040939517FA0F2E0895BF1BBB27BA0B4E
:102EC000620B730B840BF6CFDEF6B3C01F930F9328
:102ED0000027192F10789F775FE340E86130710574
:102EE0008407950718F000680E949517912B6F933F
:102EF0007F938F939F930E941B18E0E7F0E03AD0F6
:102F00005F914F913F912F910E94FC11002351F04E
:102F10002BED3FE049EC5FE300E8902717FD506898
:102F20000E9424170F911F9108959B01AC019FE30C
:102F300080E8772766270C941A139A95BB0F661FB3
:102F4000771F881F11249923A1F08823B2F79F3F90
:102F500059F0BB0F48F421F4002011F460FF04C0C5
:102F60006F5F7F4F8F4F9F4F881F9795879597F97A
:102F700008955CC0FF92EF92DF92CF92BF926B01F7
:102F80007C01B59016D0B590BB2069F09F938F93CC
:102F90007F936F93B601C7010CD02F913F914F9152
:102FA0005F910E941A13BF90CF90DF90EF90FF9037
:102FB000089545D002C09601A701EF93FF930E94A8
:102FC000FC11FF91EF913BD0EF93FF930E942417E8
:102FD000FF91EF91BA9479F70895052E092607FA23
:102FE000440F551F5F3F79F0AA27A51708F051E05D
:102FF0004795880F991F9F3F31F0BB27B91708F0FD
:1030000091E0879508959F919F91112419CF97FB87
:10301000880F991F9F3F31F0BB27B91708F091E047
:10302000879508959F919F9111240ACF662777274E
:103030008827992708959B01AC010C94FC115591A8
:08304000459135912591089599
:1030480055555555555555AAAAAAAAAAAAAAFFFF81
:10305800FFFFFFFFFFFFFFFFFFFFFFFF232340628C
:103068004570696C657073792056657273696F6E07
:1030780020302E363023000D0A01540000000000D5
:10308800000A015000000000000A0005400000008E
:10309800000A000015000000000A000000540000AB
:1030A800000A000000015000000A0000000005406E
:1030B800000A000000000015000A017102DA0F4939
:0C30C80040960200000000000000000024
:00000001FF
